:020000040000FA
:10000000D8230020150200001D0200001F0200007E
:100010002102000023020000250200000000000071
:1000200000000000000000000000000027020000A7
:1000300029020000000000002B0200002D02000039
:100040002F0200002F020000FD0A00002F02000016
:100050002F0200002F0200002F0200002F020000DC
:10006000B90A00002F0200002F0200002F0200003A
:100070002F0200002F0200002F0200002F020000BC
:100080002F0200002F0200002F0200002F020000AC
:100090002F0200002F0200002F0200002F0200009C
:1000A0002F0200002F0200002F0200002F0200008C
:1000B0002F0200002F0200000000000000000000DE
:1000C0002F0200002F0200002F0200002F0200006C
:1000D0002F0200002F0200002F0200002F0200005C
:1000E0002F0200002F0200002F020000000000007D
:1000F000000000002F020000000000002F0200009E
:1001000000000000000000000000000000000000EF
:1001100000000000000000000000000000000000DF
:1001200000000000000000000000000000000000CF
:1001300000000000000000000000000000000000BF
:1001400000000000000000000000000000000000AF
:10015000000000000000000000000000000000009F
:10016000000000000000000000000000000000008F
:10017000000000000000000000000000000000007F
:10018000000000000000000000000000000000006F
:10019000000000000000000000000000000000005F
:1001A000000000000000000000000000000000004F
:1001B000000000000000000000000000000000003F
:1001C000000000000000000000000000000000002F
:1001D000000000000000000000000000000000001F
:1001E000000000000000000000000000000000000F
:1001F00000000000000000000000000000000000FF
:10020000DFF80CD000F07EF90048004735140000FC
:10021000D82300200648804706480047FEE7FEE74F
:10022000FEE7FEE7FEE7FEE7FEE7FEE7FEE7FEE7A6
:10023000DD0800000102000040EA01039B0703D033
:1002400009E008C9121F08C0042AFAD203E011F815
:10025000013B00F8013B521EF9D270470FB400B5C4
:1002600089B00BA800906A4603480A9900F040F94B
:1002700009B05DF814FB0000580000202DE9FF5F75
:100280001D464FF0FF3BD5E9014691465F464FF0D2
:100290000008A9697F1C01988847296A8246884717
:1002A0000028F6D1BAF1FF3F0CD024F4C064002E30
:1002B00019DD600614D5BAF12B0F09D0BAF12D0F54
:1002C0000ED103E0584604B0BDE8F09F44F48064CA
:1002D000A9697F1C01988847761E8246002E02DDA0
:1002E000BAF1300F03D0B9F1000F26D032E0A9697E
:1002F000761E44F400747F1C019888478246002EC5
:1003000005DDBAF1780F06D0BAF1580F03D0B9F174
:10031000000F10D01EE0B9F1000F02D0B9F1100F9C
:1003200018D1A969761E24F400747F1C01988847AF
:100330008246102002E0082000E00A20814609E001
:1003400008FB0908A969761E44F400747F1C019813
:1003500088478246002E05DD4946504600F0BAF82F
:100360000028EDDAE96901988847A00502D46FF00A
:100370000100A8E7E00725D1600613D5600502D586
:10038000C8F1000000E0404629680A1D2A6009689B
:10039000220501D5087015E0220701D5088011E07B
:1003A00008600FE02868011D29600068210502D55A
:1003B00080F8008006E0210702D5A0F8008001E067
:1003C000C0F8008038467EE72DE9FF5FD2E901A73B
:1003D0004FF00008916999461446DDF838B046465A
:1003E00001988847054659EA0B0005D009E0A16944
:1003F000761C019888470546216A284688470028C8
:10040000F5D1681C03D05FEACA7005D015E04FF043
:10041000FF3004B0BDE8F09F2068011D2160D0F8D6
:1004200000800AE05FEACA7001D108F8015BA169A7
:10043000761C7F1E019888470546002F1ADD681C30
:1004400018D0B9F1000F0DD0E81705EBD0604211BC
:1004500020F01F0059F822102A1A01209040014272
:10046000E0D107E0BBF1000FDCD1216A28468847C4
:100470000028D7D0E16901988847BBF1000F07D168
:10048000002E05DD5FEACA7002D1002188F8001055
:10049000A068B84203DDBBF1000F03D017B16FF0C5
:1004A0000100B6E73046B4E730B50B460146002000
:1004B0002022012409E021FA02F59D4205D303FA26
:1004C00002F5491B04FA02F52844151EA2F10102A7
:1004D000F1DC30BD3A2800D2303820F02002412A29
:1004E00001D3A2F13700884201D34FF0FF307047AB
:1004F000024B9361024BD36100F032B8DD0F000074
:1005000045050000064C074D06E0E06840F0010399
:1005100094E8070098471034AC42F6D3FFF774FE16
:100520006C2600008C260000094910B508784C1C88
:1005300018B1401E0870205C10BD00210720ABBE22
:10054000207010BD02490878421C0A7070470000F4
:10055000600000200268114413780160184670475B
:10056000D1600449516104491162002111611146B1
:1005700000F00AB8550500007D050000C0B24FF438
:10058000F05100F097B900002DE9F34F8BB04FF018
:10059000000801F10C000C464FF0010B46460DF12E
:1005A000080A01906269012101989047051E2DD02B
:1005B000252D2CD0216A8847C0B16269012101989C
:1005C0009047216A88470028F7D1411E6269019847
:1005D000904700E0761CA1690B988847216A8847FC
:1005E0000028F7D1E1690B988847DBE7A1690B98F0
:1005F00088470746A84201D1761CD3E7E1690B98EA
:1006000088477F1C02D1B8F1000F6FD046E1002768
:1006100062693D463946019890472A2804D16269AB
:100620000121019890470125DFF884926269012138
:1006300001989047A0F130010A290AD24F45E5DC24
:1006400007EB870100EB4107303FDFD445F0100591
:10065000ECE7E90601D46FF000476C280AD04C287B
:1006600014D0682815D06A280DD074281CD07A2898
:100670001AD01DE062690121019890476C2802D0D0
:1006800045F0040514E045F002050DE045F02005B5
:100690000AE06269012101989047682802D045F07C
:1006A000080505E045F4006562690121019890475D
:1006B000C4E9015765283DD019DC58287AD00CDCF4
:1006C000452837D004DC252826D0412831D131E017
:1006D00046282FD047282CD12CE05B2877D06128E2
:1006E00028D063287CD0642823D15AE0D0E06F283A
:1006F00048D008DC66281DD067281BD0692821D087
:100700006E2816D127E0702845D0732868D0752848
:1007100047D078280DD14DE0A1690B988847054650
:1007200025283FF469AFE1690B9888476D1C3FF4B9
:100730006AAFB3E023466A466FF001000B99AFF34E
:1007400000809EE045F040006060A80723464FF01F
:10075000000236D43EE0E8077FF447AF2068011D71
:1007600021600068290501D506701BE7290701D51E
:10077000068017E7A90703D5F117C0E9006111E763
:1007800006600FE745F040006060A80723464FF081
:10079000080216D41EE040F60E0125EA0100606052
:1007A00016E045F040006060A80723464FF00A02BB
:1007B00007D40FE045F040006060A80708D5234645
:1007C00010226FF001000B99AFF3008059E007E0B1
:1007D000234610226FF001000B99FFF74FFD50E008
:1007E0004FF000094F464B46632802D05B2806D0E5
:1007F00040E0E80601D40120A06001273AE06269E8
:100800000121019890475E2805D14FF001096269E6
:10081000494601989047216939B900210A46534653
:1008200043F82120491C0829FADBB0B3216969B9D2
:10083000C11700EBD16253110AEB830122F01F02B2
:10084000821A01200B68904003430B60626901210A
:10085000019890475D28E8D1B9F1000F09D0002038
:10086000514651F82020D24341F82020401C08284E
:10087000F7DB02AB224600976FF001000B99FFF700
:10088000A3FD00280CDA401C08D1BBF1000F05D0F5
:100890004FF0FF300DB0BDE8F08FFFE74046F9E7BD
:1008A000E90701D108F1010806444FF0000B79E691
:1008B000CCCCCC0C7F2801D9002208E0064A02EB00
:1008C0005002C007127800D1120902F00F02012075
:1008D00090400840704700002C26000030B54FF0D3
:1008E000805000228300D0F83011C3F80C21C3F8E7
:1008F0001021624B1A60624B1B68624C2360604B94
:100900001B1D1B68241D23605D4B08331B68241DC1
:1009100023605B4B0C331B68241D2360584B103342
:100920001B68241D2360564B14331B68241D236051
:10093000534B18331B68534C20342360504B1C33EB
:100940001B68241D23604E4B20331B68241D23602D
:100950004B4B24331B68241D2360494B28331B68F1
:10096000241D2360464B2C331B68241D2360444BFD
:1009700030331B68434C40342360414B34331B6895
:10098000241D23603E4B38331B68241D23603C4BE1
:100990003C331B68241D2360394B40331B68241DE6
:1009A00023600124082902D1D0F8343113B1082979
:1009B00004D006E0354B3449196005E0D0F83431F5
:1009C00013B1082904D006E0314BFB21196005E082
:1009D000D0F8343113B1082908D00EE090F858321D
:1009E0002C48016863F30301016002E0D0F8343160
:1009F0001BB929494FF40070086028480168C907ED
:100A000002D06FF0010101602548016841F47001D6
:100A10000160BFF34F8FBFF36F8F4FF01021D1F8FC
:100A20000002002803DBD1F80402002822DA1D4B63
:100A30001C601D480468002CFCD01224C1F8004240
:100A40000568002DFCD0C1F8044201680029FCD0E3
:100A50001A6001680029FCD0BFF34F8F10487C3822
:100A60000168124A01F4E06111430160BFF34F8F46
:100A700000BFFDE70F490E48086030BD3805004053
:100A80000404001020C50040488103008C5600403B
:100A900018F50040E40E004040960240000400407B
:100AA00088ED00E004E5014000E401400400FA059F
:100AB0000090D0035C00002010B50E4C20466279F7
:100AC000017900782AB10A460146607801F042FBBC
:100AD00001E001F017FB2079401CC0B22071E178E1
:100AE000884201D9A078207103490020C1F8400153
:100AF00010BD000010000020008000400148006888
:100B0000004700002C0000200FB4054B10B503A9CE
:100B1000044A029800F018F810BC5DF814FB0000BD
:100B2000151000005400002002E008C8121F08C180
:100B3000002AFAD170477047002001E001C1121F5E
:100B4000002AFBD1704700002DE9FF4F8BB09A4679
:100B50000F460546002606E025280BD052460D9983
:100B600090476D1C761C28780028F5D10FB03046D0
:100B7000BDE8F08F0024A0460122604900E0044354
:100B800015F8013F203B02FA03F00842F7D128781C
:100B90002E2817D115F8010F44F004042A280ED08E
:100BA0006FF02F022878A0F1300109290AD808EB4C
:100BB000880102EB410100EB01086D1CF2E757F8D8
:100BC000048B6D1C287869283ED006DC0028CDD027
:100BD00063280BD0642804D136E0732810D0752820
:100BE0004BD052460D999047761C85E017F8040BC0
:100BF0008DF8000000208DF80100E946012003E097
:100C000057F8049B4FF0FF3061074FF0000401D408
:100C10000AE0641C44450DDA8442FADB19F804103A
:100C20000029F6D106E0641C8442FCDB19F80410AC
:100C30000029F8D1264404E019F8010B52460D9919
:100C40009047641EF8D257E001CF4FF00A0B0028FE
:100C500002DA40422D2102E0210504D52B218DF836
:100C60002410012103E0E10705D02021F7E70DF171
:100C7000200908910CE00021F9E701CF4FF00A0BA1
:100C8000F9E75946FFF710FC01F1300209F8012D90
:100C90000028F6D1ADEB090000F1200B600701D46C
:100CA0004FF00108D84502DDA8EB0B0000E0002062
:100CB0008046002406E009A85246005D0D99904741
:100CC000641C761C08988442F5DB04E03020524610
:100CD0000D999047761CB8F10001A8F10108F5DCE8
:100CE00005E019F8010B52460D999047761CBBF1AF
:100CF0000001ABF1010BF4DC6D1C34E709280100A5
:100D000072B609480068C00700D000BEBFF34F8F1D
:100D10000548E4380168054A01F4E06111430160C7
:100D2000BFF34F8F00BFFDE7F0ED00E00400FA05D0
:100D30000EB500210091CDE901106A4644F2010090
:100D4000FFF7DEFF0EBD10B58268C368934203D083
:100D500000F04DF9002010BD052010BD29B112B1E1
:100D6000531E134203D0092070470E2070470160C4
:100D7000838000218160C1600846704710B5826899
:100D8000C3689A1A83889A4203D800F03AF900207F
:100D900010BD042010BD000070B50A4E01460A487F
:100DA000B578FFF7D0FF04464DB10020B070711C3C
:100DB0000122C81D00F00AFD08B1FFF7B9FF204667
:100DC00070BD000034000020B4030020F0B5244EB4
:100DD00089B01F460D00044672603FD0A88829687C
:100DE00082B22048FFF7BAFF002835D1A889A96848
:100DF00082B21C481030FFF7B1FF00282CD120220E
:100E000019496846FFF718FA60690690207C00B11E
:100E100001208DF814008DF81C70607C00B10E204C
:100E20008DF81500E0680290A0680390206801909A
:100E3000606800900A480D4A6946083000F092FC4C
:100E4000002809D1B0702068401C05D00449012257
:100E5000491CC81D00F0BAFC09B0F0BD0720FBE733
:100E600034000020B40300200C260000D122000032
:100E700010B501461048FFF781FF040019D10F4853
:100E80000F4A0178515C19B1001D00F0D5FF02E056
:100E90000C3000F0B9FE60B9084907480839FFF77F
:100EA00052FF30B9054901220839044800F09EFC80
:100EB0000446204610BD0000C40300203C00002072
:100EC0001800002000F002B800F008B872B602481E
:100ED0000168491C01607047500000200349086800
:100EE000401E086000D162B670470000500000202C
:100EF00070B5054608680C46411C04D000F0FAFCA9
:100F0000206800F0C7FC6068411C02D0002100F09E
:100F1000AFFC2968A069C1F82405607D227D29689D
:100F20001043C1F86C05D4E900122868C0F81425F4
:100F3000C0F80C15207D012814D1A068411C02D0F6
:100F4000002100F095FCE068411C04D000F0D2FCC8
:100F5000E06800F09FFCD4E902122868C0F8082578
:100F6000C0F8101570BD70B5054608680C46411CE8
:100F700004D000F0C9FC206800F096FC6068411CB9
:100F800002D0002100F07DFC2968A069C1F8240589
:100F9000607D217D2A680843C2F86C05D4E90012FF
:100FA0002868C0F80C15C0F81425207D012814D13C
:100FB000A068411C02D0002100F063FCE068411CE5
:100FC00004D000F0A1FCE06800F06EFCD4E902124D
:100FD0002868C0F80825C0F8101570BD08B5684627
:100FE000FFF7DAFE0528FAD09DF8000008BD8268F8
:100FF00083881A4003689A5C0A708168491C816082
:101000007047C26883881A4003689954C168491CB4
:10101000C160704710B50446C0B2FFF729FF2046F3
:1010200010BD000070B501F0BDF815490860002042
:101030000446050201F0B6F8641C2843E4B2042C0F
:10104000F7D30F49083908600D49082010390860A6
:10105000091D0C4808600A490020103108600A4D3B
:10106000FE205FF00004287001F09CF82919641C30
:10107000E4B24870FE2CF7D301482038056070BDFB
:1010800024150040FF0004036402002008B511A0ED
:10109000FFF73AFD69461CA0FFF7E0F89DF8000055
:1010A000303802280FD89DF8001018A0FFF72CFD4B
:1010B0009DF80010174831290AD00121017011A0B4
:1010C000FFF722FD08BD072110A0FFF71DFDE1E796
:1010D0000021F3E7456E74657220646174612072CB
:1010E00061746520282731273D31204D6269742FB6
:1010F0007320616E64202732273D32204D6269746F
:101100002F73293A0D0A00002563000025630D0A9C
:10111000000000000000002008B51AA0FFF7F4FC52
:10112000694628A0FFF79AF89DF800003038072894
:101130000FD89DF80000FFF79BFE9DF80010224895
:10114000303907291BD2DFE801F0080A1012141603
:1011500018000720FFF78CFEE2E7042100E00021E1
:1011600041701AA0FFF7D0FC08BDFC21F8E7F82178
:10117000F6E7F421F4E7F021F2E7EC21F0E7FF21B4
:10118000EEE70000456E746572206F7574707574BB
:1011900020706F77657220282730273D2B3420641C
:1011A000426D2C202731273D302064426D2C2E2E9D
:1011B0002E2C2737273D2D33302064426D293A0DE0
:1011C0000A00000025630000000000200D0A000056
:1011D00010B514A0FFF798FC15A0FFF795FC24A00C
:1011E000FFF792FC2BA0FFF78FFC30A0FFF78CFCE1
:1011F00039A0FFF789FC3FA0FFF786FC43A0FFF76B
:1012000083FC4AA0FFF780FC4EA0FFF77DFC59A0AD
:10121000FFF77AFC5CA0FFF777FCBDE810405FA009
:10122000FFF772BC55736167653A0D0A0000000054
:10123000613A20456E746572207374617274206324
:1012400068616E6E656C20666F722073776565707D
:101250002F6368616E6E656C20666F7220636F6EBF
:101260007374616E7420636172726965720D0A0035
:10127000623A20456E74657220656E642063686111
:101280006E6E656C20666F722073776565700D0AEF
:1012900000000000633A2053746172742054582097
:1012A000636172726965720D0A000000643A20453C
:1012B0006E7465722074696D65206F6E2065616360
:1012C00068206368616E6E656C2028316D732D39FE
:1012D000396D73290D0A0000653A2043616E63651C
:1012E0006C2073776565702F636172726965720D2A
:1012F0000A0000006D3A20456E74657220646174C6
:101300006120726174650D0A000000006F3A20537D
:1013100074617274206D6F64756C617465642054BF
:101320005820636172726965720D0A00703A204537
:101330006E746572206F757470757420706F776548
:10134000720D0A00733A205072696E7420637572D0
:1013500072656E742064656C61792C206368616EBF
:101360006E656C7320616E6420736F206F6E0D0A62
:1013700000000000723A20537461727420525820A9
:1013800073776565700D0A00743A20537461727446
:101390002054582073776565700D0A00783A205301
:1013A0007461727420525820636172726965720DA3
:1013B0000A00000070B50D46044600684FF48871BD
:1013C00000F0C2FA4FF49071206800F0BDFA4FF4BB
:1013D0009271206800F0B8FA4FF4A271206800F012
:1013E000B3FA20681249C0F8041320686907000B9B
:1013F00040B2090E002806DA00F00F0000F1E020EC
:1014000080F8141D03E000F1E02080F8001420684B
:101410000121000B40B200F01F0291404009800002
:1014200000F1E020C0F88012C0F8001170BD00008B
:10143000100302008CB00024724801272646076082
:1014400080042546C0F80041C0F80070D0F80011B3
:101450000029FBD018226C4901A8FEF7EDFE6B486D
:10146000CDE907076A4809904FF400700A900723F6
:10147000684A07A901A8FFF7A9FC08B1FFF758FCC3
:1014800065A0FFF741FB4FF0E0214FF48070A846C4
:10149000C1F8000162B65D4DED1E07A961A0FEF71F
:1014A000DDFE9DF81C00613818286DD2DFE800F0E1
:1014B0000C1D3133496C6C6A6C6C6C6C4D6C505506
:1014C0006C585D606C6C6C6557A0FFF71DFB4F4955
:1014D00063A0491CFEF7C2FE6868502801D8014687
:1014E00026E060A0FFF710FBEEE767A0FFF70CFB1C
:1014F00046495BA0491DFEF7B1FEA868502804DCF0
:101500006868002801DBA96812E056A0FFF7FCFA22
:10151000EBE7012440E069A0FFF7F6FA3B4950A051
:101520000931FEF79BFEE868401E632805D2E96892
:101530006FA0FFF7E9FA344626E06FA0FFF7E4FA60
:10154000E9E700F0FFFD00261EE0FFF79FFDF2E750
:10155000022472A0FFF7D8FA2AE0FFF7DDFDEAE7E0
:10156000052474A0FFF7D0FA44E000F073FC0BE010
:10157000032473A0FFF7C8FA26E0042473A0FFF742
:10158000C3FA2AE0FFF724FE062C86D2DFE804F037
:101590000304101C253280E7A87818B100F0D2FDB2
:1015A00085F802802A792978687800F0D3FD1EE05A
:1015B000A87818B100F0C6FD85F802802A7929784C
:1015C000687800F085FD12E0287B00902B7A2A795C
:1015D0002978687800F0D6FD12E0A87818B100F0FC
:1015E000B1FD85F802802979287800F08BFD264628
:1015F000002452E72B7B2A7A2979287800F092FD83
:10160000AF70F4E700D00040EC250000030000209C
:1016100064000020BF220000524620546573740D00
:101620000A00000025630000456E74657220737423
:10163000617274206368616E6E656C202874776FC8
:1016400020646563696D616C206469676974732CDB
:1016500020303020746F203830293A0D0A00000005
:10166000256400004368616E6E656C206D7573744F
:10167000206265206265747765656E203020616E3A
:10168000642038300D0A0000456E74657220656E66
:1016900064206368616E6E656C202874776F2064C7
:1016A0006563696D616C206469676974732C2030AF
:1016B0003020746F203830293A0D0A00456E746569
:1016C000722064656C617920696E206D73202874C6
:1016D000776F20646563696D616C20646967697404
:1016E000732C20303120746F203939293A0D0A00CB
:1016F00025640D0A0000000044656C6179206D7559
:101700007374206265206265747765656E20312090
:10171000616E642039390D0A000000005458206DB4
:101720006F64756C6174656420636172726965725F
:101730000D0A000052582053776565700D0A0000AD
:1017400054582053776565700D0A00005258206385
:101750006F6E7374616E7420636172726965720D6D
:101760000A000000F0B505460478154889B0164611
:1017700040F82420124A08690832A2F10C0742F806
:101780002400487F385520226846FEF755FD049412
:101790002878385C48B10EB10A4A00E00022694658
:1017A000281D00F049FA09B0F0BD0EB1064A00E06C
:1017B0000022694605F10C0000F0F4F8F3E70000A0
:1017C0001C000020C92400007123000030B40378FD
:1017D000054CE35C1BB130BC001D00F063BA30BCAB
:1017E0000C3000F049B900001800002030B4037834
:1017F000054CE35C1BB130BC001D00F0D5BA30BC19
:101800000C3000F0AFB90000180000202DE9FF41B6
:101810001C46DDE90A7815460E46684600F04EF88B
:1018200046EA450141EA840141EA072242EA0841C9
:10183000009A00EB8200C0F80017BDE8FF812DE997
:10184000FF411C46DDE90A7815460E46684600F061
:1018500043F846EA450141EA840141EA072242EAA7
:101860000841009A00EB8200C0F80017BDE8FF8134
:101870001CB500220B46009211460192FFF7C6FFED
:101880001CBD1CB500220B46009211460192FFF7C9
:10189000D6FF1CBD1CB5002100910B460122019111
:1018A0001146FFF7B3FF1CBD1CB5002100910B468C
:1018B000012201911146FFF7C2FF1CBD01682029DA
:1018C00002D24FF0A040704701F01F0101600148B3
:1018D00070470000000300500168202902D24FF039
:1018E000A040704701F01F010160014870470000EF
:1018F0000003005001B56846FFF7E0FF009A0121A0
:101900009140C0F8081508BD01B56846FFF7E4FF2F
:10191000009A01219140C0F8081508BD40580028E0
:1019200000D00120704708B5002242504058009076
:1019300008BDD0F80403084000D00120704740588B
:10194000002800D00120704708B5002242504058BE
:10195000009008BD0121B1EB507F01D101207047FB
:101960000020704770B50D4600F094FB04000FD0C6
:101970000020FFF7A7FA207920B10020FFF7A4FA92
:10198000112070BD0120256020710020FFF79CFA16
:10199000002070BD0149024800F002BD6403002030
:1019A000002000402DE9F0410546007916460F461B
:1019B00000EB40012D4A01EBC00102EB810494F8D9
:1019C0002A1011B10820BDE8F081294951F82010F2
:1019D0002868FFF7C7FF08B11120F4E73946284609
:1019E000FFF786FA66603869206030004FF0010624
:1019F0002FD03F7F4FF48E712868FFF794FF4FF48C
:101A0000A2712868FFF78FFF28681A49C0F80413ED
:101A100028684FEA4711000B40B2002806DA00F0B0
:101A20000F0000F1E02080F8141D03E000F1E02039
:101A300080F800142868000B40B200F01F0206FA7C
:101A400002F14009800000F1E020C0F88012C0F8E7
:101A5000001128680421C0F800150020A061E06191
:101A600084F8290044F8140FA675ACE7640300203D
:101A700004260000800002002DE9F05F0546007991
:101A80004FF4017600EB400303EBC000344B03EB53
:101A900080040020636813B12B68C3F80863A3694E
:101AA0004FF000096BB1E06938B1606810B1286887
:101AB000C0F804631120BDE8F09FE26101202161BC
:101AC00005E0C4F82490A261E160C4F81C9094F889
:101AD0002910014302D1284600F0A4FB60680028C9
:101AE000286803D0C0F804630020E4E74FF4A2762E
:101AF0003146FFF718FFB2464FF4927B59462868EB
:101B0000FFF70CFF06464FF484712868FFF706FFC5
:101B1000804651462868FFF701FF074648EA07005C
:101B20003043EBD056EA070007D12146286800F081
:101B300049FBA169606A8142E0D8C4F818900EB1EF
:101B40000320B8E70FB10F20B5E794F82910012062
:101B50000029296801D00860C6E74860C4E7000092
:101B6000640300202DE9F047054600790B4600EBA1
:101B7000400101EBC000234901EB8004284600F03E
:101B800043F810B11120BDE8F0874FF00008C4F809
:101B90002080A360626184F828804FF48E764746E7
:101BA00031462868FFF7BFFE28684FF00109C0F8EA
:101BB00008902146286800F065FB606800BBD5F8F6
:101BC00000A00EE094F8280008B10F2716E0314677
:101BD0005046FFF7A3FE0028F4D02146504600F0FF
:101BE00051FB216A60698142F1D331462868FFF7D1
:101BF00095FE0028F9D02868C0F80C90C4F814802D
:101C00003846C0E764030020007900EB400101EB97
:101C1000C000044901EB80004069002800D0012089
:101C200070470000640300200149024800F064BCD2
:101C300090030020002000402DE9F04105461646A3
:101C400000790F46154A00EBC00102EB810494F8BD
:101C5000201011B10820BDE8F081114951F8201081
:101C60002868FFF77FFE08B11120F4E739462846BF
:101C7000FFF779F96660386920601EB1397F284620
:101C8000FFF798FB28680821C0F800150020A06124
:101C9000E0610121606184F82010DCE790030020FE
:101CA000082600002DE9F05F044600790E4600EB9F
:101CB000C001DFF8F0A017460AEB81053046FFF7B8
:101CC00049FEB0B168684FF000084FF4047910B1D4
:101CD0002168C1F80893A8694FF0000B80B1E8694A
:101CE00048B1686810B12068C0F804931120BDE8BD
:101CF000F09F1020FBE7EF614FF001082E6102E03A
:101D0000EE60C5E9067B00254FF488712068FFF777
:101D10001BFE4FF4A2712068FFF716FE2068C0F882
:101D20003465C0F838752068B8F1000F12D0D0F8CB
:101D3000001241F02001C0F800122079D04600EBDB
:101D4000C0010AEB8100406838B12068C0F80493F4
:101D50002846CCE701210160EFE74FF4887A4FF481
:101D6000A27951462068FFF7EAFD074649462068F8
:101D7000FFF7E5FD06464FF492712068FFF7DFFD9F
:101D8000014647EA06000843EBD0227902EBC20382
:101D900008EB8302C2F818B001B10325002ED7D09A
:101DA0000F25D5E7900300202DE9F04704460E46A5
:101DB0000079204900EBC00001EB80051746304652
:101DC000FFF7C8FD30B1204600F036F820B11120F1
:101DD000BDE8F0871020FBE76F61AE604FF49076AE
:101DE000002731462068FFF7AFFD4FF4AC7841463D
:101DF0002068FFF7A9FD2068AA686969C0F8442532
:101E0000C0F84815206801218160686878B9B1463A
:101E100049462068FFF793FD064641462068FFF7D4
:101E20008EFD0643F4D000B10F27002068613846CC
:101E3000CEE70000900300200079054900EBC000C8
:101E400001EB80004069002800D0012070470000AD
:101E50009003002010B521A0FEF756FE234C2078F9
:101E600010B1012805D101E021A000E029A0FEF772
:101E70004BFE6078F42829D007DC78B104280BD019
:101E8000EC2827D0F0280CD122E0F8281CD0FC2820
:101E900018D0FF2805D11FE027A000E02EA0FEF7F4
:101EA00033FE35A06168FEF72FFE3AA0A168FEF769
:101EB0002BFE3FA0E168FEF727FEBDE8104043A0DF
:101EC000FEF722BE43A0EAE74AA0E8E751A0E6E712
:101ED00058A0E4E75FA0E2E766A0E0E75061726126
:101EE0006D65746572733A0D0A00000000000020F1
:101EF0004461746120726174652E2E2E2E2E2E2E5A
:101F00002E2E2E2E3A2031204D6269742F730D0A29
:101F1000000000004461746120726174652E2E2EF1
:101F20002E2E2E2E2E2E2E2E3A2032204D62697409
:101F30002F730D0A00000000545820506F7765720F
:101F40002E2E2E2E2E2E2E2E2E2E2E2E3A202B34B0
:101F50002064426D0D0A0000545820506F7765725E
:101F60002E2E2E2E2E2E2E2E2E2E2E2E3A2030209F
:101F700064426D0D0A0000002853746172742920B8
:101F80004368616E6E656C2E2E2E2E2E3A202564CF
:101F90000D0A0000456E64204368616E6E656C2E0C
:101FA0002E2E2E2E2E2E2E2E3A2025640D0A0000C7
:101FB00054696D65206F6E20656163682063686198
:101FC0006E6E656C3A2025640D0A0000206D730D5D
:101FD0000A000000545820506F7765722E2E2E2E66
:101FE0002E2E2E2E2E2E2E2E3A202D342064426D93
:101FF0000D0A0000545820506F7765722E2E2E2E39
:102000002E2E2E2E2E2E2E2E3A202D382064426D6E
:102010000D0A0000545820506F7765722E2E2E2E18
:102020002E2E2E2E2E2E2E2E3A202D313220644290
:102030006D0D0A00545820506F7765722E2E2E2E8B
:102040002E2E2E2E2E2E2E2E3A202D31362064426C
:102050006D0D0A00545820506F7765722E2E2E2E6B
:102060002E2E2E2E2E2E2E2E3A202D323020644251
:102070006D0D0A00545820506F7765722E2E2E2E4B
:102080002E2E2E2E2E2E2E2E3A202D333020644230
:102090006D0D0A000349884201D1034870470020B2
:1020A00070470000002000402C000020074800215D
:1020B000C0F80012C0F8101101220261D0F81021FE
:1020C000002AFBD0C0F8101170470000001000403B
:1020D00070B514460D460646FFF7E8FFFEF7A2FF6F
:1020E00006480721C0F8001205490E60091D0D6061
:1020F0000349091F0C600121016070BD0010004000
:102100000C15004010B50C46FFF7D0FF0348012125
:10211000C0F80012024A1460416010BD0010004077
:102120000815004030B40446054804708170017100
:10213000C2700021417130BC184600F083B8000025
:1021400010000020024901204860FFF7AFBF0000E7
:102150000080004070B514460D460646FFF7A6FF06
:1021600006480121C0F80012054A1660121D1560CC
:10217000034A121F1460016070BD0000001000408F
:102180000C15004030B4064C029D60702170A270A6
:102190002271E37001206071284630BC00F052B813
:1021A0001000002005480021C0F80011D0F80011EF
:1021B0000029FBD0024800687047000000D00040B2
:1021C00008D5004070B5054688690C4600284FF4D4
:1021D000847128460AD0FFF7A6FBD5F81805626A75
:1021E000E1688854606A401C606270BDFFF79BFB29
:1021F000D5F8180570BD1FB501238DF80030CDE965
:102200000121D0E90012684690471FBD1FB5012388
:102210008DF800308DF808100192D0E90012684660
:1022200090471FBD10B5044600684FF49271FFF748
:102230007AFB4FF484712068FFF775FB2068012159
:10224000016010BD0D4910B501224A60C1F800229D
:102250000B4C002323600223241D2360084C04231D
:102260000C3423601304C1F804334FF47A7310FB69
:1022700003F0034B3C3318600A6010BD008000403F
:102280000485004070B50C4605464FF48E71FFF78B
:102290004AFB216AA068415C206A401C2062C5F8A4
:1022A0001C1570BD1FB500228DF8002002918168B9
:1022B00001914261D0E90012684690471FBD017844
:1022C000022901D0012902D14068FEF731BD7047D3
:1022D0007CB50178244D81B301290BD002292BD183
:1022E0008DF80010C068691C01900122C81DFFF71D
:1022F0006DFA2EE0406801781C48FEF73FFD1B4C4C
:10230000012618B18DF80060019006E0A068E16830
:10231000814205D000208DF8000069686846884732
:10232000A068E168081AA188884207D80E490122EE
:10233000491CC81DFFF74AFA7CBD01E0AE70FBE7FF
:102340000A4809491030FEF7FEFC30B103208DF831
:102350000000696868468847EEE70349012201F1F9
:102360000800FFF743FAE7E734000020B403002039
:102370001FB50A4601788DF8001041680191017A75
:102380008DF80810C0680390044850F822100838EF
:1023900050F82220684690471FBD0000240000200E
:1023A0002DE9FF470C4605464FF40071FFF7C1FACF
:1023B00001274FF40178002618B34FF4927949466B
:1023C0002846FFF7ABFAE0B149462846FFF7ABFADB
:1023D000C5F8088394F8290000B96F6002208DF8D1
:1023E0000000D5F88004C5F880040390A06902902D
:1023F000E0680190A661E661D4E900126846904762
:1024000028E004212846FFF794FA18B34FF48471AA
:102410002846FFF783FAE8B121462846FFF7D2FEA7
:10242000616AA069884215D1E06938B1E268616AE1
:10243000A0612069E6616662E06008E094F8290026
:1024400000B96F60C5F80883A661E268616A20463A
:10245000FFF7D1FE4FF48E7841462846FFF75EFA2B
:1024600078B1206A6169884202D294F8280020B3CA
:1024700041462846FFF757FA616911B12046FFF738
:1024800011FF4FF4A27841462846FFF747FA00288B
:1024900018D041462846FFF746FA94F8290000B1C3
:1024A0002F60A06900280DD0A661E268616A04B0BF
:1024B0002046BDE8F047FFF79EBE21462846FFF7BD
:1024C000E1FEDEE7BDE8FF871FB50A4601788DF81B
:1024D000001041680191017A8DF80810C0680390DE
:1024E000044850F82210083850F8222068469047D7
:1024F0001FBD0000240000202DE9FF410C464FF4D1
:10250000927705463946FFF71AFA0026C0B13946D8
:102510002846FFF719FA02208DF80000D5F880044C
:10252000C5F880040390D5F83C058DF80800E068F4
:102530000190A661E661D4E900126846904723E065
:102540004FF4887739462846FFF7F9F9E0B1394664
:102550002846FFF7F9F9D5F83C15A069884213D150
:10256000E06960B1E268D5F8000220F02000C5F80B
:102570000002E069A0612069E661E06001E0A66117
:10258000E2682046FFF742FE4FF4A277394628461C
:10259000FFF7D5F960B139462846FFF7D5F9A069AC
:1025A00030B1A661D5F83C152046E268FFF72EFE53
:1025B0004FF4907739462846FFF7C1F9002813D029
:1025C00039462846FFF7C0F9606900280CD0D5F8D5
:1025D0004C058DF800608DF80800A06801906661D8
:1025E000D4E9001268469047BDE8FF81080000006A
:1025F00006000000050000000700000000000000C9
:1026000000E0D70195190000291C0000FFFFFFFF23
:10261000FFFFFFFFFFFFFFFFFFFFFFFF00000000C6
:10262000000000000000D60107010000DDDDDDDD57
:10263000DCBBBBDDDDDDDDDDDDDDDDDD9888888853
:1026400088888888777777777788888885555556FA
:102650006666666666666666666888888333333251
:1026600022222222222222222228888D8C26000049
:102670000000002064000000280B0000F02600008D
:102680006400002074230000380B000001000000EB
:1026900000000000500000000A00000000000000E0
:1026A000000000000000000000000000000000002A
:1026B000000000000000000000000000000000001A
:1026C00000000000000000000000000000200040AA
:1026D000000000000020004000000000000000009A
:1026E00000000000000000000090D0030000000087
:0400000500000201F4
:00000001FF
